:020000040000FA
:100000008A01C701C601FD2AF000030E8301F10039
:100010000A08F2008A010B115E30C51B583E8100B0
:10002000C51F16280830BB06BB1D1928A40A2C3092
:10003000A7073B08071A103A1039031D23283B1D58
:10004000BB0A65215E29071A2728871F2A28640012
:10005000BC17BB0628088207532997299C299F298A
:10006000A7296521BB133B1DBB17F2238207532928
:10007000A8035B292A0E0F3982070F34073407348F
:1000800003340334013401340034003401340134C6
:1000900003340334073407340F34311AAB290F30DB
:1000A00031058207202BEF2A5A2C5A2C5A2C5A2C15
:1000B0003F2C3F2C5A2C5A2C432C412C5A2C5A2C76
:1000C0005A2C452C30083E06031D6F282F084B067E
:1000D000031D6F283108C039803A031992282F0870
:1000E000031D4F2BF0303005703A031D4F2B29298B
:1000F0003C1C83283C103C1783168C24A201B2239D
:10010000A00134229422451130082F0403199228AB
:1001100030083D06031D62282F084A06031D622889
:10012000C5184515CE010630A9001F24B108031DCE
:100130004510C801C80AB10E310CB10E073982074B
:100140004D28BD2CCF2CCF2C142D212D4E2BC80A81
:10015000311AF028C80A45195A2C3208BF00310854
:1001600003392225D200FF3A03195A2C3308B20072
:10017000B10C310C033982075A2CD728DC28C0284F
:10018000C51E5A2C3208392182075A2CD3285D0803
:10019000CC210B30D2000301CC211130B921DF3941
:1001A000CC002222452C5D08CC21452CD200BA215E
:1001B00032060319452C5A2C32080739C200C20AEC
:1001C000C1010314C10DC20BE228BA21C200321AC8
:1001D000222941084205B21941060319452C5A2C1F
:1001E000310807398207FB28FB28FB28FB28022956
:1001F0000429D628D6284607451C143EBF004708C8
:1002000022251B2911301B29B203BF010310B20D97
:10021000BF0DB20DBF0DB11D12293208C6003F0837
:10022000C700452C32084606031D5A2C3F084706D6
:10023000031D5A2C452CD200FF3A03195A2CB11D2C
:10024000D728C028C51E5A2C41084204B21D4106B9
:10025000C3280630A9004514CE011F24C51E4F2B0C
:100260003208B3003108B2003008B100AD18AA2836
:10027000F028DD00F6305206FE390319003452082A
:10028000093C031D4C29C0305D02031C0034E830DA
:100290005D020318003401345208003C031D013490
:1002A000DD1F02340034A801C5171230AD00AE01C5
:1002B0002F308400A80AF830BB05BB0A72088A00F8
:1002C000710E8300F00E700E0900CF1F69293C18D3
:1002D000080026082702031C0800A700A10AA10A9B
:1002E0004F1E832954085302031C8329C83021025E
:1002F000031C8329E830210203183C1992291F1599
:10030000BC143C1592293C11CF1E8E294F080F3981
:100310005402031C8E29230895000800230821029B
:10032000031C942995010800FF30950008003B1933
:100330005329AD0B5B295A293B19A80A5B293B1DA0
:100340005329C51356308102FE30AC005A29BB0A2E
:10035000A80A65215E29C80A0E303105023A031D3C
:100360005A2CB213311CB2170B30D2003208CC21F8
:100370005A2CD200F630520603198534F730520653
:1003800003190D348312520803178D0083160C14C1
:1003900083120C08031308008B13640083120317E5
:1003A0008C000313520803178D0083160C158C1351
:1003B00055308D00AA308D008C148C18DD290C115D
:1003C000031383128B17E8290130A500C030C50044
:1003D0000630B921C300C30DC30D83304304A6000A
:1003E0001D30B921CF000730B921D300D30D1E3005
:1003F000B921D7001F30B921D8002030B921D90048
:100400001130B921CC00CC1E0E2A0A30B921BE0011
:10041000BD000930B921CB00CA00142ACB01CA01A2
:100420000030B921BE00BD00C5100B30B921C3009A
:100430004512C31B45167F3903190800BD00CA01C8
:10044000C51408001130D2004C08CC210800C000AF
:100450000830C1004008C001BF0C0318C007C00C21
:10046000C10B2C2ABF0C08002008031D392AD40117
:1004700008004C1E4C2ABF001B3027222530C00725
:100480004008B921C2004003B921C300420227221B
:1004900040084307D4000800C4010430B921DC003F
:1004A000FE390319FF30BF00DC000310BF0C013020
:1004B000B921DB00C2000310C20C4208BF072008AC
:1004C0002722420840020318672AC40A003CBF00E2
:1004D0008030200203186F2A003CC40AC417272268
:1004E000BF0D400D4418003CC3002008BF00003C75
:1004F00027220530B921FE39031D812A5B08DC075C
:100500005C0CBF000310BF0C40082722BF0DC00DBC
:10051000BF0D400DC307C31B902A430D013E4A2A5D
:100520000030C41FFF304A2A5408031D4F1EEC2A16
:1005300053025408031CEC2ABC1C08001F190800B5
:10054000C4011E020318A62A4414003CBF00BF0ABF
:100550005708272254080F3C4008031CBB2AF030E0
:100560004005031DBA2AF030BF05BF0EC00E40057E
:100570003F04BB2AFF304418C12A5502031C030163
:10058000C42A55070318FF30D500C4015408BF0022
:10059000C0005908C0020318540827221E08400250
:1005A0000318D42A4414003CBF0058082722F03016
:1005B0004005031DE22AF030BF05BF0EC00E400506
:1005C0003F04E32AFF304418E92A55070318FF3097
:1005D000EC2A5502031C0030A300BC1008000B30AD
:1005E000D2000301CC210230CC0022220301D20A26
:1005F000CC210030D2000330CC21831603178C139A
:1006000003130E0883128B13C200C401CF1B0D2BE2
:10061000871B0D2B071E062B4416C21C162B4218D7
:10062000202BA53050060319482BD006BC01CD0164
:10063000CD17A001CF1B1E2B4408BC048030BB008B
:100640008B133F30AB00A2013030BC05E4210030F9
:10065000B92103192D2B031A3F2B64004C1D3F2B8E
:100660003C14CF1B482BCD133C0810394406BC1E4C
:100670003C2B03193D2B482BBC06A209482BD40167
:10068000A301D501A101A401850186018701CE0145
:1006900083160E148E148C24B2233422A801AD01CB
:1006A0002F308400AE01B301B4013B138B160B1144
:1006B0008B17C1233B1B78280830B9210319592B0C
:1006C0004E02031C592B0A2DAA0A0319CE0A183010
:1006D000AB0540302A058338AB04AB122B1FAB1699
:1006E0003A202A05031D2B1506302A0503192B1065
:1006F00078302A050319AB10D10B822BAB13230CD6
:10070000FF3CD100C3010530C4000130C1004108E5
:100710004D050319952B44081D3CB9212B05031DDC
:10072000952B4408183CB921C3040310C10DC40B18
:10073000872B0030C306431C861243188616C31C41
:100740000612C3180616431D861143198615C31DCC
:100750000611C3190615431E8610431A8614080095
:10076000BC1D0800BC113C1ABA2B87122B160717A8
:10077000AB11BE2B0713AB1587162B122208D60020
:1007800008003C1CC52BBC1F640050302402031C15
:10079000F02BA4006423A90BCE2B4510A50BF02B46
:1007A000200856020319EC2B031CDC2BA00A023094
:1007B000B921A5000E30E12BA0030330B921A5001B
:1007C0000F30B921BF007F39BF1B003CA507031DB7
:1007D000EB2B5608A0003422A50AA0080319B02369
:1007E000942200343B0DBB1E022CBB12031C022CB6
:1007F0004517AE08031D00340430AD02031C00345D
:10080000AD0A3B17AC0D03180134BB163B1B00347B
:100810002C08AE06451F152C4513C039C03A0319E4
:10082000142CAF01840AAD0A2C088000840AAD0A9A
:1008300007302D0203180034AC01AC090134C51691
:100840002F083506031DC512B50630083606031DF0
:10085000C512B60631083706031DC512B7063208A1
:100860003806031DC512B80633083906031DC51224
:10087000B90634083A06031DC512BA06080022223A
:10088000452CCC163F2CCC123F2C451C5A2C8B13DC
:100890002030C1000713871686160616FF30950014
:1008A0006400C201C20B522CC10B502C9501861260
:1008B00006124E2B4808AD020319502B031C4E2B79
:1008C0003208B1003308B2003408B300C80B602C02
:1008D0009928BC16BC11451D702C451A3F06722C78
:1008E0004C183F063F05031D792C3C12AB197C2C9C
:1008F00008003C162B1E0800BC15CD1BB2230800B7
:100900000D30B921451D0330FF3ACD05FF3A311EA8
:100910000301CD0431120800C93081000E309F0060
:10092000FF30920003178C01031383120C309700E1
:100930000430920081309F008B013C18AB2C831651
:1009400001308500C1308600903087008312850118
:10095000860187010800831601308500CF308600AC
:100960009030CF1FB42CFF308700831230308600C8
:100970000030850004308700080031083F3A031D2D
:100980005A2CC80A8030BF0032086924320DFE3963
:1009900003190B2DFE3E03190A2DFE3EFD2CC51139
:1009A0002030BF0031086924CC1C80241F30B105E1
:1009B00031080F3903190B2DFF3E03190A2D0310BF
:1009C000B10DB11A3114B112490831020318EA2CE1
:1009D000C515023EFF3EC4003108C900FC3EBF0001
:1009E00097302722C00E3F0E40060F394006C4083C
:1009F000031DFD2CC51DF63E053E3C1BBC1D042DF4
:100A0000BC111030BC060C2D013EA200CD1BA00075
:100A1000CD130D2DA0013C13A2012208BC19030126
:100A2000D600342294225A2CCC188024C330CD0511
:100A30000C30B921451DFF30B105B10D310D3C39E8
:100A4000CD045A2C0339031DFF3406303F0203182E
:100A50002B2D063E080008303F020318312DF83ECA
:100A6000080008303F02031CFF34FD3E03183A2DF6
:100A7000093E080010303F02031CFF34FD3E0318FE
:100A8000432D0C3E080014303F02031CFF34FB3E94
:100A900003184C2D113E08001C303F02031CFF348C
:100AA000FE3E0318552D133E080020303F02031C64
:100AB000FF34FB3E03185E2D183E080030303F0225
:100AC000031CFF34F43E0318672D243E0800423017
:100AD0003F02031CFF34E43E0318FF34403E08008D
:084000000000000000000100B7
:02400E00763DFD
:10420000030001000500050001004B000000FF0055
:10421000000000000000000000000000000000009E
:104220000100160000000100020004000800100058
:104230001000080000000000000030008000800036
:10424000A6000000000000000100020003000500BD
:1042500008000C00100015001A00210027002F0094
:1042600037004000490053005E006900750081007E
:104270008F009C00AB00BA00CA00DA00EB00FF0020
:00000001FF
